:1000000017C1000031C100002FC100002DC1000048
:100010002BC1000029C100000C9402090C941109A5
:1000200023C1000021C100001FC100001DC100004C
:100030001BC1000019C1000017C1000015C100005C
:1000400013C1000011C100000FC100000DC100006C
:100050000BC1000009C1000007C1000005C100007C
:100060000C94ED090C94F809FFC00000FDC00000DD
:10007000FBC00000F9C00000F7C00000F5C00000A0
:10008000F3C00000F1C00000EFC00000EDC00000B0
:10009000EBC00000E9C00000E7C00000E5C00000C0
:1000A000E3C00000E1C00000DFC00000DDC00000D0
:1000B000DBC00000D9C00000D7C00000D5C00000E0
:1000C000D3C00000D1C00000CFC00000CDC00000F0
:1000D000CBC00000C9C00000C7C00000C5C0000000
:1000E000C3C00000C1C00000BFC00000BDC0000010
:1000F000BBC00000B9C00000B7C00000B5C0000020
:10010000B3C00000B1C00000AFC00000ADC000002F
:10011000ABC00000A9C00000A7C00000A0C4000040
:10012000A3C00000A1C000009FC000009DC000004F
:100130009BC0000099C0000097C0000095C000005F
:1001400093C0000091C000008FC000000C946209B1
:100150008BC0000089C0000087C0000085C000007F
:1001600083C0000081C000007FC000007DC000008F
:100170007BC0000079C0000077C0000075C000009F
:1001800073C0000071C000006FC000006DC00000AF
:100190006BC0000069C0000067C0000065C00000BF
:1001A00063C0000061C000005FC000005DC00000CF
:1001B0005BC0000059C0000057C0000055C00000DF
:1001C00053C0000051C000004FC000004DC00000EF
:1001D0004BC0000049C0000047C0000045C00000FF
:1001E00043C0000041C000003FC000003DC000000F
:1001F0003BC000000C94D3130C948B140C040E041D
:10020000100412041404160418041A04C50BEB0B92
:10021000120C3B0C440C490C8E0C930CB20CB90C18
:10022000550C5D0C650C700C720C740C7C0C840C01
:1002300011241FBECFEFCDBFDFE2DEBF10E2A0E092
:10024000B0E2E8E3FBE202C005900D92AA3BB107E1
:10025000D9F72DE2AAEBB0E201C01D92AC3FB20784
:10026000E1F791D20C949A15CBCE84E0809356009E
:100270008CE1BDD3809363008BEB8093660080E8B4
:100280008093650081E08093600088ED84BF1092C8
:10029000410083E080935000809151008330E1F76A
:1002A0008091500081608093500088E180935500D8
:1002B0008091510080FFFCCF80915000806180933D
:1002C00050008091510084FFFCCF88ED84BF84E012
:1002D000809340000895E0E7F0E085818E7F85837C
:1002E000E0E0FAE08FEB9DE586A397A380EE9EE227
:1002F00080A391A382E0808308958091200A909149
:10030000210A813E2EE2920718F020919E2306C01A
:10031000803E2EE2920721F020919B2320936A00D9
:1003200020910520222321F080910520815033C0A7
:10033000885F9A42813D974080F11092BA20809167
:10034000BB209091BC20A091BD20B091BE20019611
:10035000A11DB11D8093BB209093BC20A093BD2014
:10036000B093BE208091BB209091BC20A091BD2075
:10037000B091BE20892F9A2FAB2FBB278093BE232D
:100380008091BB209091BC20A091BD20B091BE2057
:100390008093BD2386E08093052080910720909173
:1003A00008200196B1F4809109208F3F91F080914F
:1003B0000620811106C0809106208150809306207E
:1003C00008958091140190911501809307209093D6
:1003D00008200895009709F45EC00CF457C040E06F
:1003E00020916B0030E020939C2330939D2320913B
:1003F0009C2330919D233695322F222737952795C0
:1004000020939C2330939D2350916A0020919C233C
:1004100030919D23250F311D20939C2330939D23E4
:10042000000020919C2330919D232817390728F440
:1004300010929C2310929D23089520919C2330912B
:100440009D23280F391F2115304238F08FEF9FE18F
:1004500080939C2390939D23089520919C23309119
:100460009D23442329F0A901481B590BCA0102C04E
:10047000820F931F80939C2390939D2380919C23B4
:1004800090919D238F7780936A000895919581952F
:10049000910941E0A5CF0895CF93DF93C091200A41
:1004A000D091210A80910320909104209E01281B65
:1004B000390B20939F233093A0238091BA20811180
:1004C0004BC080919F239091A0238E3C9F4FD4F4EA
:1004D00080919F239091A0238B369F4F9CF0809119
:1004E0000220882321F080910220815008C0809151
:1004F0006A0080939E2381E08093BA208CE08093F1
:1005000002202AC08CE08093022080919F2390914A
:10051000A0238A369F4F1CF08FEF9FEF02C081E02F
:1005200090E08093992390939A2380919F239091B8
:10053000A0232091992330919A2360E370E00E94D8
:100540007115261B370B2093992330939A238091A2
:10055000992390919A233EDF8091BA20813029F52A
:1005600080919F239091A023C39794F080910220C3
:10057000882331F08091022081508093022015C0A1
:1005800080916A0080939B2383E08093BA200DC002
:1005900080919F239091A023873991051CF481E0DD
:1005A00090E002C08FEF9FEF15DFC0930320D09340
:1005B0000420DF91CF9108958617970779F0681787
:1005C000790728F49C01261B370BB90109C086174F
:1005D000970718F4681B790B03C0089560E070E07A
:1005E000CB010895CF93DF9380910020909101205B
:1005F000892B51F0809100209091012001978093E8
:1006000000209093012043C080E490E0809300207C
:100610009093012080910720909108200196B9F1D4
:10062000809114019091150120910920263018F431
:1006300067E771E002C06EEE72E00E945D15EC01AA
:1006400080910720909108208C179D0758F46091A5
:10065000072070910820CE01AFDF029718F080ECE0
:100660009DE511C08091072090910820C817D907F7
:1006700070F46091072070910820CE019DDF0297F1
:1006800030F08FEB9DE58093360A9093370ADF9127
:10069000CF910895AC01460F571F861B970B2091F1
:1006A000200A3091210A24173507C8F72091200A23
:1006B0003091210A8217930790F70895E0E8F6E059
:1006C0008FE0808385E0848308951F93CF93DF9329
:1006D000C0E4D0E0198180E4898340E250E064ED19
:1006E0007DE280E290E00E94200F1983DF91CF919C
:1006F0001F9108951F93CF93DF93C0E4D0E0198139
:1007000080E4898387ED97E20E94560F81E00E9482
:10071000680F1983DF91CF911F91089508950F936A
:100720001F93842F50E0415851099DE7949F9001F9
:10073000959F300D112490910920953048F484380C
:1007400010F029583E4F9091C42067E771E004C033
:100750009091C4206EEE72E0969FA001979F500D7D
:100760001124420F531F4850584D0FE813E02DE756
:1007700030E060E00E9410131F910F9108951CBE9D
:10078000EEEFF0E40994A1DF8091D42D882369F085
:1007900080E2E4EDFDE2A7EDB7E201900D928A95CB
:1007A000E1F71092D727A6DFEADF87E08093A20067
:1007B00078945BDDB3DF77D765D188D160E080E0E6
:1007C0001FD10BD18CE0FFD03BD5DFD5F8D576DF3C
:1007D00060EA70E28AEA93E20E949315000000004A
:1007E0000000000000000000000000000000000009
:1007F00000000000000000008091BF20882371F3FA
:10080000E091D6258E2F90E088309105A0F4FC0170
:10081000E250FF4F0C94841584D10DC0F2D10BC06F
:1008200077D209C0F9D207C083D305C007D403C06B
:1008300006D401C075D41092BF20D0CF089508957A
:10084000809114018093B323809115018093B42388
:10085000809124018093B523809125018093B62354
:100860008091200A8093BF238091210A8093C02326
:1008700080911401909115018634914080F080910F
:10088000140190911501893A914048F48091140126
:10089000909115018093F42D9093F52D0000809197
:1008A000C220882339F017DD1092C22081E08093A6
:1008B000C12008958091C120882341F08091BA2001
:1008C000833019F41ADD8EDE01C0E6DD8091C02090
:1008D000882351F080911401909115018093F42D9B
:1008E0009093F52D1092C020809109202091140141
:1008F00030911501853028F481E02737314030F000
:1009000004C081E02E3E324008F080E08093C42095
:1009100008950F931F9381E08093C7208093C22096
:100920000FE813E02DE730E048EF57E260E081E8A0
:100930000E9410132DE730E045E758E260E082E8BE
:100940000E9410132DE730E042EF58E260E083E8A8
:100950000E9410132DE730E04FE659E260E084E892
:100960000E9410132DE730E04CEE59E260E085E87C
:100970000E9410132DE730E049E65AE260E086E875
:100980000E94101381E01F910F9108951092C720CB
:10099000089581E0089581E0089510922002982F33
:1009A0009C7193689093200287FF03C080E192E0DE
:1009B00002C080E090E0892B8093210210922202F5
:1009C000109226020895E0E0F2E010AA836880AB5E
:1009D00080E181AB12AA16AA0895E0E0F2E010A629
:1009E00083E880A78FE281A712A616A60895AAEC35
:1009F000B1E092E09C93E82FF0E084911C9208957E
:100A0000909171009D7F909371001092000262306E
:100A100011F09CE101C09EE19093010290E490935B
:100A20000202811102C080E401C080EC80930302C5
:100A3000613011F084E001C083E08093040280E221
:100A4000D6DF80930C0281E2D2DF80930D021092F8
:100A500018021092190281E080930002BECF1F920B
:100A60000F920FB60F9211248F9300000000000028
:100A7000000081E0809323028F910F900FBE0F90B2
:100A80001F901895CF93DF93E0E7F0E082818B7F92
:100A90008283C0E2D3E08DE0888380E4898389E0AB
:100AA0008A8383E3A4DF888782E3A1DF898787E3E2
:100AB0009EDF8A8786E39BDF8B87E0E2F6E080811A
:100AC000836080831482DF91CF910895E0E7F0E0A6
:100AD00080818E7F808383E8809300010895E0E029
:100AE000F1E0108A80E4808B10A280A310AA80AB72
:100AF000E0E4F1E0108280831092C6201092C520BD
:100B00001092C4201092A8231092A9231092A62319
:100B10001092A72308958093D62581E08093BF206B
:100B20000895CF93DF9310920920D9DFC0E0D1E080
:100B30001EAA84E288AB19AA49E54AAB32E03BAB76
:100B400060910B2070910C206CAB7DAB67ED75E272
:100B500068AF79AF1AAE9BE39CAF93E09DAF1EAE3A
:100B600028A9206828AB10924601E0E4F1E08083D8
:100B700010924101409342019093430140910D2016
:100B800050910E20409344015093450146EC53E2AE
:100B9000409348015093490110924A0129E3209360
:100BA0004C0190934D0110924E019081906890837A
:100BB000188A90E4988B888B198A95E99A8B90E132
:100BC0009B8B4EEE52E04C8B5D8B888F398F1A8E4B
:100BD00088EF97E28C8F9D8F1E8E68EC70E084EF1B
:100BE00091E058DD88EC90E08093072090930820F6
:100BF00081E08093062088898068888BDF91CF917F
:100C000008951F93CF93DF9311E01093092067DFBE
:100C1000C0E0D1E018AA80E488AB84E088AB19AAD0
:100C20001AAA4BE44BAB1CAA1DAA1EAA8AE090E2AA
:100C300088AF99AF1AAE60EA6CAF38E03DAF1EAE38
:100C400088A9806A88ABE0EAF8E085E58083808344
:100C500010924601E0E4F1E084E2808310924101C9
:100C600099E59093420122E020934301A0910B204B
:100C7000B0910C20A0934401B0934501A7EDB5E2DB
:100C8000A0934801B093490110924A019BE39093CD
:100C90004C0193E090934D0110924E019081906829
:100CA000908388A319A295E99AA34BA34EEE52E034
:100CB0004CA35DA368A739A71AA666EE7AE26CA7D3
:100CC0007DA71EA6888B198A9A8B90E19B8B4C8BF3
:100CD0005D8B888F298F1A8E88EF97E28C8F9D8F7E
:100CE0001E8E68EC70E084EF91E0D4DC88EC90E03C
:100CF00080930720909308201093062088A1806895
:100D000088A388898068888BDF91CF911F9108958F
:100D10001F93CF93DF9312E010930920E0DEC0E031
:100D2000D1E01EAA84E288AB19AA39E53AAB1BAB25
:100D300040910B2050910C204CAB5DAB47ED55E240
:100D400048AF59AF1AAE9BE39CAF93E09DAF1EAE88
:100D500028A9206828AB10924601E0E4F1E08083E6
:100D600010924101309342019093430120910D2054
:100D700030910E20209344013093450126EC33E25C
:100D8000209348013093490110924A0129E32093AE
:100D90004C0190934D0110924E0190819068908388
:100DA000188A90E4988B888B198A45E94A8B90E1E0
:100DB0009B8B2EEE32E02C8B3D8B888F198F1A8EF9
:100DC00068EF77E26C8F7D8F1E8E88A319A24AA3ED
:100DD0009BA32CA33DA384E388A719A71AA686EE9C
:100DE0009AE28CA79DA71EA668EC70E084EF91E0C4
:100DF00051DC88EC90E0809307209093082081E0FC
:100E00008093062088898068888B88A1806888A361
:100E1000DF91CF911F9108951F93CF93DF9313E03C
:100E2000109309205CDEC0E0D1E010924601E0E4BE
:100E3000F1E084E280831092410129E52093420190
:100E400092E09093430140910B2050910C204093ED
:100E500044015093450147ED55E2409348015093BA
:100E6000490110924A019BE390934C0110934D016C
:100E700010924E019081906890831EAA88AB19AAA7
:100E80002AAB1BAB20910D2030910E202CAB3DAB3B
:100E900026EC33E228AF39AF1AAE99E39CAF1DAF11
:100EA0001EAE98A9906898AB18A250E458A394E09D
:100EB00098A319A21AA24BE44BA31CA21DA21EA226
:100EC0002AE030E228A739A71AA630EA3CA728E092
:100ED0002DA71EA698A1906A98A395E59093A008C7
:100EE000188A588B888B198A85E98A8B4B8B8EEEF2
:100EF00092E08C8B9D8B388F298F1A8E88EF97E22A
:100F00008C8F9D8F1E8E68EC70E084EF91E0C2DBC9
:100F100088EC90E0809307209093082081E08093F4
:100F2000062088898068888BDF91CF911F91089572
:100F30001F93CF93DF9314E010930920D0DDC0E01E
:100F4000D1E018AA80E488AB18AB19AA1AAA3BE42E
:100F50003BAB1CAA1DAA1EAA8AE090E288AF99AFFB
:100F60001AAE50EA5CAF88E08DAF1EAE98A9906AC9
:100F700098AB95E59093A00810924601E0E4F1E06B
:100F800094E290831092410129E52093420122E0EE
:100F90002093430160910B2070910C2060934401D9
:100FA0007093450167ED75E26093480170934901C4
:100FB00010924A012BE320934C0123E020934D0132
:100FC00010924E01208120682083988B198A45E970
:100FD0004A8B3B8B2EEE32E02C8B3D8B588F898FCA
:100FE0001A8E68EF77E26C8F7D8F1E8E98A319A200
:100FF0004AA39AE49BA32CA33DA393EC98A789A7AB
:101000001AA686EE9AE28CA79DA71EA668EC70E051
:1010100084EF91E03FDB88EC90E080930720909391
:10102000082081E08093062088898068888B88A1C9
:10103000806888A3DF91CF911F910895FFCFCF9350
:10104000DF9386E0809309204ADDC0E0D1E01EAA4C
:1010500084E288AB19AA39E53AAB93E09BAB4091A7
:101060000D2050910E204CAB5DAB46EC53E248AFE7
:1010700059AF1AAE29E32CAF9DAF1EAE28A9206848
:1010800028AB10924601E0E4F1E080831092410128
:101090003093420122E02093430140910B20509174
:1010A0000C20409344015093450147ED55E2409395
:1010B00048015093490110924A013BE330934C019F
:1010C00090934D0110924E01908190689083188A00
:1010D00090E4988B888B198A95E99A8B90E19B8B89
:1010E0004CED55E04C8B5D8B888F298F1A8E88EFE5
:1010F00097E28C8F9D8F1E8E68EC70E084EF91E0FC
:10110000C9DA80E991E0809307209093082081E07C
:101110008093062088898068888BDF91CF9108951D
:10112000CF93DF9387E080930920D9DCC0E0D1E042
:101130001EAA84E288AB19AA39E53AAB93E09BABCF
:1011400040910D2050910E204CAB5DAB46EC53E22C
:1011500048AF59AF1AAE29E32CAF9DAF1EAE28A9F8
:10116000206828AB10924601E0E4F1E08083109201
:1011700041013093420122E02093430140910B2032
:1011800050910C20409344015093450147ED55E2A6
:10119000409348015093490110924A013BE3309338
:1011A0004C0190934D0110924E0190819068908374
:1011B000188A90E4988B95E2988B198A95E99A8B16
:1011C00090E19B8B4CED55E04C8B5D8B888F298F8C
:1011D0001A8E88EF97E28C8F9D8F1E8E68EC70E0E0
:1011E00084EF91E057DA80E991E0809307209093B3
:1011F000082081E08093062088898068888BDF91B1
:10120000CF9108951F920F920FB60F9211248F93D2
:1012100081E0809303018F910F900FBE0F901F907C
:1012200018951F920F920FB60F9211248F9382E0A0
:10123000809303018F910F900FBE0F901F90189510
:10124000E0E7F0E083818C7F838384818C7F8483DB
:1012500080818D7F8083E0E8F1E080EC82831286DC
:1012600088EC81831186A0E0B8E034E03C9323E071
:1012700011962C93119714961C92149785ED91E07A
:1012800096968D939C93979716961C921697E0E4EA
:10129000F8E030832183148286A397A31682E0E6C8
:1012A000F6E0808180618083E0E4F9E083E181837E
:1012B000148282E08683A6A3B7A310A611A681E0BC
:1012C000808308951F920F920FB60F9211242F93CF
:1012D0003F934F935F938F939F93CF93DF931F928F
:1012E000CDB7DEB78FEF80934C098091092087300E
:1012F00031F480912C02898390912D0202C090914B
:101300002C028091C320891B2091680930916909C2
:1013100082308CF02A3F374070F420916809309178
:10132000690989301CF481E090E002C086E090E019
:10133000820F931F18C020916809309169098F3F6F
:10134000B4F42730310598F020916809309169098B
:10135000883F1CF081E090E002C086E090E0A901A7
:10136000481B590BCA0180937809909379090F9013
:10137000DF91CF919F918F915F914F913F912F91ED
:101380000F900FBE0F901F901895E0E7F0E083815B
:101390008F7E8383E0E4F6E080818A6A80838FEF2A
:1013A000848388E5828BE0EAF8E080E3838384EC41
:1013B000858387E08683178288E184830895E0E748
:1013C000F0E08381877F8383E0ECF8E0118288E599
:1013D0008093550680E6808308951F920F920FB682
:1013E0000F92112400000F900FBE0F901F901895C0
:1013F0001F920F920FB60F9211248F93EF93FF93CA
:10140000E0EAF8E080818083FF91EF918F910F9067
:101410000FBE0F901F9018959FB7F894A0E5B0E00D
:1014200016968C911697897F16968C931697E0E600
:10143000F0E080E885838BEB868316968C91169777
:10144000846016968C938081816080839FBF08950D
:101450009FB7F894E82FF0E0E059FF4F6095808146
:10146000682360839FBF0895CF93863011F0C0E05A
:1014700001C0C8E18091510081FD0DC09FB7F89473
:10148000809150008260809350009FBF80915100F6
:1014900081FFFCCFC1DF6C2F636084E490E0B5D4A2
:1014A00060E480E0CF91D4CF8091C82008958091EE
:1014B000C820813009F46ACA0895F0D0FC01838104
:1014C0008093C820811101C024CA81E008959091C1
:1014D000C625892F807697FF07C0803491F48091CC
:1014E000C72581110EC057CA803459F48091C72591
:1014F000811107C08091CC259091CD25892B09F0D1
:1015000048CA80E008958091C8258F770C949A127C
:101510009091D020911102C080E00895E091CD20FB
:10152000F091CE200190F081E02D94818917A0F7F1
:10153000E093CB20F093CC20228133812E0F3F1FEC
:10154000E217F30798F49181943061F49281891342
:1015500009C09381691306C0E093CB20F093CC209F
:1015600081E008959081E90FF11DEACFE093CB204F
:10157000F093CC20D1CFE091CD20F091CE200190FE
:10158000F081E02D228133812E0F3F1FFC0140812D
:10159000E40FF11DE217F30748F48181843031F044
:1015A000853039F08081E80FF11DF4CF80E090E0C4
:1015B0000895CF0108951F93CF93DF93182FA8DFCD
:1015C000882339F1C091CB20D091CC20CE01D3DF3C
:1015D000EC01892B41F04C815D816B818A81B7D709
:1015E0008111F4CF16C0E091CD20F091CE209281F0
:1015F0008381E92FF82FE10FF11DE10FF11D01901B
:10160000F081E02D0190F081E02DDF91CF911F91CD
:10161000099480E0DF91CF911F910895EF92FF929E
:101620001F93CF93DF93C82F60E072DF811102C058
:1016300010E02DC0E091CD20F091CE2092818381E9
:10164000E92FF82FEC0FF11DEC0FF11DE080F18078
:10165000D7011696ED91FC9117970995682F8C2F5D
:1016600057DF182F882321F3C091CB20D091CC20B5
:10167000CE0181DFEC01892B21F08A810E94BA130F
:10168000F7CFD7011296ED91FC9113970995812F11
:10169000DF91CF911F91FF90EF9008958091CB2023
:1016A0009091CC200895DBC6CF938091D0208823E1
:1016B00011F0C0E008C01092D0201092D4201092F7
:1016C000D520CF910895E091CD20F091CE200190CA
:1016D000F081E02D8481C81770F78C2F9FDFCF5FDA
:1016E000F2CFCF938091D0208823F1F0C0E0E09139
:1016F000CD20F091CE20A081B18114968C91C81795
:1017000098F492818381E92FF82FEC0FF11DEC0FF3
:10171000F11D0190F081E02D0084F185E02D3097DE
:1017200009F00995CF5FE3CFCF9108950F931F93F1
:10173000CF93DF931092D0251092D1251092D2250D
:101740001092D3251092D4251092D5258091C625CC
:1017500087FF07C02091CC253091CD25232B09F49C
:101760004EC3982F9076903409F00BC1E091C725B5
:101770008E2F90E0FC01E05AF109EA30F10508F003
:10178000CBC2EA5FFE4F0C94841581E08093C020A9
:1017900080910720909108208093B72380910720A3
:1017A000909108209093B82380919E238093B92331
:1017B00080919B238093BA2380916A008093BB23FE
:1017C00080916B008093BC236091CC257091CD25D6
:1017D0008AEA93E2D4C0109200088091C8259091C3
:1017E000C92580933608909337088091CA258F7059
:1017F000809300086091CC257091CD2586EC93E212
:101800009FD68091CC259091CD2520910D203091AF
:101810000E208217930709F4BDC280930D20909388
:101820000E2026C0109240088091C8259091C925AD
:1018300080937608909377088091CA258F70809363
:1018400040086091CC257091CD2587ED95E278D642
:101850008091CC259091CD2520910B2030910C20AA
:101860008217930709F496C280930B2090930C2063
:101870008091092051C010926809109269098091E5
:10188000C8258093C32086C28091C82580932406F2
:1018900081C2E091C825F091C925E830F10508F032
:1018A0003BC2E05FFE4F0C94841560E080E0A8D856
:1018B0008091CA2572D880E02FC060E080E0A0D877
:1018C0008091CA256AD881E027C061E081E098D87C
:1018D0008091CA2562D88091CB2575D882E01CC042
:1018E00083E01AC084E018C060E080E089D880916D
:1018F000CA2553D885E010C061E080E081D880918E
:10190000CA254BD886E008C062E080E079D8809193
:10191000CA25806842D887E0FED83CC28091C8259D
:101920008093840637C28091C8259091C925892B60
:1019300091F00E94650380E2E4EDFDE2A7EDB7E2DD
:1019400001900D928A95E1F781E08093D7270E945C
:101950007A030E946503E9E7F0E091E088EDF894EE
:1019600084BF90836091CC257091CD258AEA90E266
:1019700006C06091CC257091CD2589EA90E2E0D532
:1019800009C29111C9C187FFFBC02091CC253091BC
:10199000CD252115310509F4BFC18F7109F09EC015
:1019A0008091C725863071F0883009F48EC081118E
:1019B000B3C12230310509F0AFC162E070E084EDBF
:1019C00090E2DDCF8091C8259091C925292F33273A
:1019D00022303105A1F060F42130310509F09CC1BD
:1019E0008091192090911A20DC016C9170E05BC00D
:1019F0002330310589F12F30310509F18DC1E09196
:101A00001920F0911A202189821708F085C19927A1
:101A1000880F991F880F991FE0911B20F0911C20BF
:101A2000E80FF91F80819181FC016281738188D563
:101A3000E091CE25F091CF2582E0818335C0809161
:101A40001D2090911E20009709F466C1DC011296BA
:101A50006D917C91139727C099278130910569F08A
:101A600038F0029709F058C168E08AE890E208C0AF
:101A700064E070E08CE990E216C067E083E990E2F0
:101A8000282FAAE7B0E2FC01819190E08D939D930D
:101A90008E2F821B8617C0F3660F6E5F60937820CF
:101AA00070E088E790E24CD58091CC259091CD25CF
:101AB0002091D0253091D1258217930708F06AC173
:101AC0008093D0259093D12565C12130310509F04F
:101AD00023C161E070E080ED90E251CF8130C1F52B
:101AE0008091C7258A3009F017C12130310509F0EE
:101AF00013C18091D020882309F40EC1C091CA255A
:101B0000D091CB250091CD201091CE20D801ED9120
:101B1000FC918481C81708F0FFC060E08C2FF8DCCE
:101B2000882309F4F9C0DD27CC0FDD1FF80182817D
:101B30009381C80FD91FE881F9810680F781E02DD4
:101B400009958093D22061E070E082ED90E217CF9A
:101B5000823009F0E1C08091C7258111DDC02230BB
:101B6000310509F0D9C08091CA253AD590E080931B
:101B7000C9209093CA2062E070E089EC90E2FFCE29
:101B80008F7109F07DC08091C725833009F4C4C0EE
:101B900018F48130A1F0C0C0853019F0893039F1D6
:101BA000BBC08091CC259091CD25892B09F0B4C084
:101BB00083E89AE08093D2259093D325EBC080915F
:101BC000CC259091CD25892B09F0A6C08091C82500
:101BD0009091C925019709F09FC08091D4209091E0
:101BE000D5208D7F8093D4209093D520D3C0809131
:101BF000CC259091CD25892B09F08EC09ED48823C9
:101C000009F48AC02091C8253091C9253327E09175
:101C10001920F0911A20818990E08217930708F427
:101C20007BC042DD8091C8259091C9258093D0204A
:101C3000882309F4AFC099278150904C880F991FD1
:101C4000880F991F20911B2030911C20820F931F19
:101C50008093CD209093CE20C0E0E091CD20F091F4
:101C6000CE200190F081E02D8481C81708F092C049
:101C700060E08C2FA0DC882309F44EC0CF5FEDCF4D
:101C80008130E9F48091C7258B3009F045C08091FF
:101C9000CC259091CD25892B09F03EC08091D02094
:101CA000882309F439C0C091CA25D091C8258C2F4A
:101CB000B5DC882389F16D2F8C2F7DDC2BC0823021
:101CC00059F58091C725813019F0833089F024C0FF
:101CD0008091CC259091CD25892BF1F48091C82558
:101CE0009091C925892BC1F48091CA2580D412C056
:101CF0008091CC259091CD25892B71F48091C825B8
:101D00009091C925892B41F48091CA2503D58091F2
:101D1000CA2539D581113EC08091C6258F71813089
:101D2000D9F58091D020882309F469C0C091CA25D3
:101D3000D091CB250091CD201091CE20D801ED91EE
:101D4000FC918481C81708F05AC060E08C2FE0DB5A
:101D5000882311F1FE01FF27EE0FFF1FD801129615
:101D60008D919C911397E80FF91F00811181D80183
:101D70001696ED91FC9117970995682F8C2FC8DB6B
:101D8000882351F0D8011496ED91FC91159709958F
:101D9000882311F081E034C08091C6258F71823094
:101DA00071F58091D020882351F1C0E0E091CD20E1
:101DB000F091CE20A081B18114968C91C817F8F4CF
:101DC00092818381E92FF82FEC0FF11DEC0FF11DAB
:101DD00000811181D8011696ED91FC911797099514
:101DE000682F8C2F95DB882351F0D8011496ED9144
:101DF000FC91159709958111CDCFCF5FD7CF80E0AA
:101E0000DF91CF911F910F9108951BBEFC0128ED2A
:101E100024BF608308958091CF0187FDFCCF089592
:101E20001F93CF93DF93C0ECD1E01A858A8761E0DE
:101E30008BEC91E0EADF1A87DF91CF911F91089533
:101E4000CF92DF92EF92FF920F931F93CF93DF9386
:101E50008C017B016A01DFDFCCECD1E088818860F6
:101E60008883B801705FA601C70154D68881877F37
:101E70008883DF91CF911F910F91FF90EF90DF90BA
:101E8000CF900895CF93DF93C82FD62FC4DFACEC4B
:101E9000B1E08C9188608C93EC2FF0E0F05FD08300
:101EA0008C91877F8C93DF91CF9108950F931F932F
:101EB000CF938C01B0DFC0E0F80161918F018C2FCE
:101EC000E1DFCF5FC032C1F7CF911F910F9108952D
:101ED000CF93C82FA0DF20E2C29FC0011124E0EC05
:101EE000F1E012829183808385E3CF9199CF409175
:101EF000CA01E62FF72F8093CA0184914093CA014B
:101F00000895E82FF0E0EA50F24D80818F3F09F408
:101F1000FFCF9FB7F89480818F5F80839FBF089524
:101F2000E82FF0E0EA50F24D8081811101C0FFCF2F
:101F30009FB7F8948081815080839FBF0895CF938D
:101F4000C82F80919823C11105C0882339F081E002
:101F5000E7DF04C0811102C081E0D3DFC093982382
:101F6000CF910895282F2F70082E000C990B392F30
:101F7000331F3327331F832F90E0820F911D820F71
:101F8000911D23E0880F991F2A95E1F78C5D9C4DE8
:101F900008950F93E8ECF4E080818F7D8083808149
:101FA0008F7D8083ECE2F3E202E0059310922E2312
:101FB00010922F2300E2069300E40693E4E2F3E29A
:101FC00000E2069300E40693E6ECF5E2148615863B
:101FD0001686178612861386109207230F9108958E
:101FE0000F9385E080930723EDE2F3E204E005938D
:101FF000E5E2F3E204E005930F9108950F9383E087
:102000008093072310922E2310922F23ECE2F3E209
:1020100002E006930F910895E091D225F091D32527
:10202000309709F009940895282F2F70082E000C7E
:10203000990B392F331F3327331F832F90E0820FE3
:10204000911D820F911D029749E0489F9001499F81
:10205000300D1124C901895A9D4D0895AF92BF9248
:10206000DF92EF92FF920F931F93CF93DF93D82EBF
:10207000DBDFEC018D2D76DF7C01DC011196EC912C
:10208000E770E150E73040F4F0E0EE0FFF1FE45559
:10209000FF4D0081118102C008E010E02D813E81DA
:1020A0008B819C814881D7FE4AC0F7016681778188
:1020B000260F371F2D833E8328173907A1F1BC0156
:1020C000621B730B9B01211574E0370738F02FEF6B
:1020D00033E0C901B801F1D4281B390B41FF0AC014
:1020E000C901B801EAD4AC0191E0452B09F090E0B8
:1020F000892F01C080E0988180FB91F99883D701F6
:1021000016961D921C92179712962D933C93139737
:1021100029813A818D819E81820F931F14968D9320
:102120009C93159708C041FF78C04D7F4883168265
:10213000178212821382F70102E0069385C0D7014D
:102140001296AD90BC90139742FF0FC0E981FA81BF
:10215000B801B3D4B0E4DB9EB001112469567F4DC1
:10216000AC01CF01820F931FD5D42D813E812A0D62
:102170003B1D2D833E838B819C818217930710F436
:102180008D839E83F70126813781A216B30609F05D
:1021900044C02D813E818217930709F43EC0AC01F3
:1021A000421B530B9A01211554E0350750F02FEFD5
:1021B00033E0C901B80181D4B901681B790BCB01A7
:1021C00007C0C901B80179D4D901A81BB90BCD0149
:1021D000F701128213828017910798F48881846036
:1021E0008883F0E4DF9EC001112489569F4DD701FA
:1021F00014968D939C93159716960D931C93179791
:102200009ACF49815A812D813E81240F351FF701D4
:1022100024833583868397838ECF888180FF14C083
:102220008E7F8883EF81F885309771F06D817E8194
:102230004D2D80E0DF91CF911F910F91FF90EF9096
:10224000DF90BF90AF900994DF91CF911F910F91D4
:10225000FF90EF90DF90BF90AF9008950F93CF93D2
:10226000DF9380910723833029F4D6DEDF91CF916D
:102270000F918FCE2091032330910423C091D0255C
:10228000D091D125C21BD30B61F58091052390918C
:102290000623820F931F809305239093062320919A
:1022A000CC253091CD258217930721F08091D6203F
:1022B000882331F084E080930723E4E2F3E236C020
:1022C000E091D425F091D525309799F00995882390
:1022D00081F01092032310920423C091D025D09155
:1022E000D125C034D10528F01092D620C0E4D0E02A
:1022F00003C081E08093D620C0932E23D0932F2358
:1023000080910323909104232091CE253091CF25F5
:10231000280F391F2093302330933123C80FD91F42
:10232000C0930323D0930423ECE2F3E202E006938C
:10233000DF91CF910F9108950F93CF938091CC04AB
:1023400080FF63C021E02093CC0484E293E2FC018F
:1023500000E80693ECE2F3E200E806932093CA0457
:10236000FC0100E1069380910723882329F0835024
:10237000823008F451DE0DDE8091262390912723D0
:10238000089709F044C088E0E3ECF2E2A6ECB5E27D
:1023900001900D928A95E1F78091C8048062809344
:1023A000C8048091C80480628093C804BFD9C82F34
:1023B000811102C015DE2BC08091C62587FF0DC09C
:1023C00010920523109206231092032310920423E7
:1023D00082E08093072342DF1BC08091CC2590913F
:1023E000CD25892B11F40ADE13C01092052310921B
:1023F0000623109203231092042381E08093072385
:10240000E4E2F3E202E0069303C0C0E001C0C1E0F1
:102410008C2FCF910F910895CF93CFB7F89481E08F
:102420008EDDEAECF4E080E4808380E28083E1ECFE
:10243000F4E0808181608083A9ECB4E08C918260BB
:102440008C93E8ECF4E08081806480838C918160DF
:102450008C93808180688083CFBFCF910895CF9384
:102460001092600080E300D88091C0048064809363
:10247000C00481E080936000CFB7F89480E090E0E2
:10248000FC0123E0EE0FFF1F2A95E1F7E85FFC4D0A
:10249000158E01968E30910599F780E090E039E035
:1024A000389FF001399FF00D1124E95AFD4D20812C
:1024B0002E7F208301968C30910591F76AE170E0C0
:1024C00082E015DD8F3F09F48FE18093FA046BE120
:1024D00070E082E00CDD8F3F09F48FE18093FB0414
:1024E0008091C00486608093C0048091C00480689D
:1024F0008093C0048091C00480618093C00484E212
:1025000093E28093C6049093C7048091C0048062D4
:102510008093C0048FEF8093C5048091C8048260CB
:102520008093C8041092982385E0EBDC75DFCFBF61
:10253000CF9108958093C30408958091C3040895B2
:10254000E6ECF5E2808791876287738708951F9391
:10255000CF93DF93162FEA0105DDFC018181807C9A
:10256000D1F5612F6370613019F020F080E803C06D
:1025700080EC01C080E4C038D105E1F050F4C032F5
:10258000D105A1F0C034D10599F06097C9F491E06C
:1025900018C0C11592E0D90779F0CF3F93E0D90771
:1025A00069F0C115D14061F495E00BC092E009C01B
:1025B00093E007C094E005C096E003C097E001C037
:1025C00090E0118226E02083982B918381818062A4
:1025D000818381E001C080E0DF91CF911F91089558
:1025E000C1DCFC01818182FB882780F90895CF93AB
:1025F000C82FB8DCFC01818182FF0FC081818B7FF5
:1026000081838C2F11DDFC01908190FF06C09E7F9D
:1026100090830780F085E02D099581E0CF910895A2
:10262000AF92BF92CF92DF92EF92FF920F931F93E0
:10263000CF93DF93D82EC62E5A017901F5DCEC0139
:102640008D2D90DC9C01DC0111968C911197807C82
:1026500009F454C011968C911197807C803C21F034
:1026600011968C9182FD4AC09FB7F894888180FFB3
:1026700002C09FBF43C0816088839FBFA982BA8286
:10268000EB82FC821D821E820F83188791E0C110AD
:1026900004C0E114F10409F090E0888190FB81F915
:1026A0008B7F8883D7FE02C0F90122C0D901119621
:1026B0008C911197807C803CC1F41196EC91E7706D
:1026C000E150E73040F4F0E0EE0FFF1FE455FF4D1E
:1026D0006081718102C068E070E0C701EED1892B92
:1026E00021F088818E7F888309C0F90112821382CC
:1026F000168217828D2DB2DC81E001C080E0DF916F
:10270000CF911F910F91FF90EF90DF90CF90BF90EE
:10271000AF900895EF92FF920F93CF93C82F22DCD2
:102720007C018C2F81DCDC01F70102E005939C9198
:1027300090FF1BC09E7F9C931796ED91FC9118977C
:10274000309799F0D701C7FF05C016966D917C911F
:10275000179704C012966D917C9113974C2F81E0CE
:10276000CF910F91FF90EF900994CF910F91FF902F
:10277000EF900895CF93C82FCDDF8C2FF3DBFC01B2
:102780001182CF9108950F93CF93C82FEBDBFC01FB
:1027900081818460818301E006938C2FBBDF81E01F
:1027A000CF910F9108951F920F920FB60F9211249F
:1027B0000F932F933F934F935F936F937F938F93D9
:1027C0009F93AF93BF93CF93EF93FF938091CB04ED
:1027D00087FF08C080E88093CA040E94710B0E94A2
:1027E000200486C08091CB0482FF18C084E08093CF
:1027F000CA0480912C2386FF7BC08091CC0481FD8C
:1028000077C09ADD811174C080910723813011F463
:10281000F5DB6EC0843009F06BC021C08091CB0421
:1028200081FF26C082E08093CA048091242386FF22
:102830005FC08091CC0481FD5BC07EDD811158C0FA
:1028400080910723823041F484E080930723E4E2FF
:10285000F3E202E006934CC0833009F049C0EDE298
:10286000F3E204E00593E5E2F3E204E0059340C0FF
:102870008091CB0484FF25C080E18093CA04C1E02D
:102880008C2F48DF8C2F806845DFCF5FC630C1F7C3
:102890000E94540B1092C30410922523C09324234A
:1028A00083E48093252310922D23C0932C238093BF
:1028B0002D2383EC92E2809328239093292369DBD4
:1028C00017C08091CB0486FF08C080E48093CA04BF
:1028D00080E035DB0E941E040BC08091CB0485FF95
:1028E00007C080E28093CA0481E029DB0E941F04B4
:1028F000FF91EF91CF91BF91AF919F918F917F9178
:102900006F915F914F913F912F910F910F900FBE5B
:102910000F901F9018951F920F920FB60F921124CF
:102920000F931F932F933F934F935F936F937F93D7
:102930008F939F93AF93BF93CF93DF93EF93FF93C7
:102940008091CC0481FF1AC082E08093CC048091F6
:10295000C5048195880FE4E2F3E2E81BF1092081C8
:1029600031812452334283E0369527958A95E1F7E9
:10297000822F869520FD06C0C0E005C0DDDC8823DF
:1029800019F386C0C0E8C80F8C2FECDAFC01208157
:1029900025FF7EC000E20693C11174C08091072319
:1029A000843019F439DBF5DA73C0009126231091D5
:1029B00027238091D0259091D125C0910323D091D8
:1029C000042398012C0F3D1F8217930718F48C01E4
:1029D0000C1B1D0B8091CE259091CF25A80163EC97
:1029E00072E28C0F9D1F96D0C00FD11FC09303239E
:1029F000D09304230034110569F48091052390914C
:102A000006238C0F9D1F2091CC253091CD25821758
:102A1000930788F0C093D025D093D125E091D42599
:102A2000F091D525309729F00995811102C0D8DAA7
:102A30002FC0E4DA2DC08091D0259091D125C81700
:102A4000D907D9F4E091D425F091D525309779F3C1
:102A50000995882361F32091052330910623809105
:102A6000032390910423820F931F80930523909357
:102A700006231092032310920423E4E2F3E202E01F
:102A8000069306C0C03811F4E9DB02C08C2FE6DAE9
:102A9000FF91EF91DF91CF91BF91AF919F918F9176
:102AA0007F916F915F914F913F912F911F910F9166
:102AB0000F900FBE0F901F901895AA1BBB1B51E1E2
:102AC00007C0AA1FBB1FA617B70710F0A61BB70B9E
:102AD000881F991F5A95A9F780959095BC01CD0143
:102AE000089597FB072E16F4009406D077FD08D0C2
:102AF000E4DF07FC05D03EF4909581959F4F089543
:102B0000709561957F4F0895EE0FFF1F0590F4912A
:102B1000E02D0994FB01DC0102C001900D924150AF
:102B20005040D8F70895FB01DC0101900D92002080
:082B3000E1F70895F894FFCFCE
:102B380040000CE02E0AFFFFFFFF55800080005D7B
:102B48000A570A670A540A000064201F2000002858
:102B58002023200F2000000009023C000101008012
:102B6800FA0904000006FFFFFF0007058101800045
:102B78000107058201800001070583018000010724
:102B8800058401800001070585018000010705868D
:102B9800018000011201000200000040EB0394BA1A
:102BA8000002010200010000000300000000000014
:102BB800000000000000000000004C6162726164C7
:102BC8006F72004573706F54656B0000040309044D
:102BD800646562756731323300010400100020001B
:0A2BE8004000800000010002FF031E
:00000001FF
